:100000000C943E000C945B000C945B000C945B0021
:100010000C945B000C945B000C945B000C945B00F4
:100020000C945B000C945B000C945B000C945B00E4
:100030000C945B000C945B000C945B000C945B00D4
:100040000C945B000C945B000C945B000C945B00C4
:100050000C945B000C945B000C945B000C945B00B4
:100060000C945B000C945B000C945B000C945B00A4
:100070000C945B000C945B000C945B0011241FBE7D
:10008000CFEFD0E1DEBFCDBF11E0A0E0B1E0EEE305
:10009000F1E002C005900D92A034B107D9F711E04C
:1000A000A0E4B1E001C01D92A034B107E1F70E94C5
:1000B0007E000C949D000C94000012B891E095B95C
:1000C0008FEF88B91BB811B894B987B91AB80895D9
:1000D0008F73E82FF0E0E050FF4F8081282F022E31
:1000E00022952025022E26952695202530E02F5F8B
:1000F0003F4F3595279520FF8064089512B891E011
:1001000095B98FEF88B91BB811B894B987B91AB8E7
:100110002898C0E0D0E005C0219680B10E94680018
:1001200088B92097C9F7189904C0289AC1E0D0E08F
:0E013000F4CF2898C1E0D0E0F0CFF894FFCFD4
:10013E002C01020304050607080924252728292275
:10014E0010131415161718122C21112C323A2C2CB0
:10015E0023343536373839330E2D201E2C2C2C1DDA
:10016E00310A320F3C302C2C2C19262C2C3E2C1CF8
:00000001FF
